:0200000480007A
:100000006F004005732F2034930F8000630AFF03B5
:10001000930F90006306FF03930FB0006302FF038A
:10002000170F0000130F8F2E63040F0067000F00DF
:10003000732F203463540F006F00400093E19153FD
:10004000171F000023203FFC171F0000232E0FFA6C
:100050006FF01FFF930000001301000093010000E8
:10006000130200009302000013030000930300003A
:100070001304000093040000130500009305000022
:10008000130600009306000013070000930700000A
:1000900013080000930800001309000093090000F2
:1000A000130A0000930A0000130B0000930B0000DA
:1000B000130C0000930C0000130D0000930D0000C2
:1000C000130E0000930E0000130F0000930F0000AA
:1000D000732540F16310050097020000938202012E
:1000E000739052307350447497020000938202015F
:1000F00073905230735000189702000093824202AE
:10010000739052309B021000939252039382F2FF3D
:100110007390023B9302F0017390023A73504030A7
:100120009702000093824201739052307350203046
:100130007350303093010000970200009382C2ECAC
:1001400073905230130510001315F501635C050020
:100150000F00F00F930110009308D0051305000065
:100160007300000093020000638A02007390521033
:10017000B7B200009B82921073902230735000300F
:10018000372500001B05058073200530970200000D
:100190009382420173901234732540F17300203032
:1001A0009301200013030000970200009382C20015
:1001B0006783220011A019A06F0000129301300084
:1001C000970200009382C200678312006F008000D4
:1001D0006F0080109301400013030000970200009D
:1001E0009382C2006783320011A019A06F00C00E75
:1001F0009301500013030000970200009382C20095
:100200006F03600011A019A06F00000D9301600042
:1002100013030000970200009382C20063030000F2
:1002200011A019A06F00400B93017000631500002E
:100230006F00C00009A009A06F00000A73601230AF
:10024000F323103093F343006386030A7370123074
:10025000F323103093F34300639E0308F3225030DE
:1002600017030000130363011303230073105330BB
:100270006F0060000100BDA87390523073601230AF
:1002800093018000F323103093F34300638403064B
:100290000100737012300100F323103093F3430018
:1002A000638C030297020000938282029382E2FF32
:1002B0007390123473701230B72300009B83038055
:1002C00073A00330730020306302000073601230AB
:1002D0006F004002631030020F00F00F63800100D6
:1002E0009391110093E111009308D005138501004B
:1002F000730000000F00F00F930110009308D00569
:100300001305000073000000130520006380A102A4
:1003100013054000638CA100130550006388A10001
:10032000130560006384A1006FF01FFBE31603FA5E
:100330009305000073252034E310B5FAF32510343B
:1003400093854500E39AB2F87325303463060500BF
:100350001305E5FFE31255F8938585007390153476
:1003600073002030731000C0000000000000000087
:10037000000000000000000000000000000000007D
:1010000000000000000000000000000000000000E0
:1010100000000000000000000000000000000000D0
:1010200000000000000000000000000000000000C0
:1010300000000000000000000000000000000000B0
:081040000000000000000000A8
:040000058000000077
:00000001FF
